:020000040000FA
:1000000000306500FF3066000515A0010530A10035
:100010003C30A20033200130A3000F200A28A01892
:100020002528861C0800A1032108031D1928053076
:10003000A10090309D004020220821079D00402013
:100040007F309D004020A0140800861808008030F2
:100050009D004020220821079D00402000309D0087
:100060004020A01008000D309C00FF309B000A309B
:100070009A009A0B39289B0B37289C0B35280800CF
:10008000051118309F009F0B432808309B009D0CE2
:1000900003184D2800000511502805150000000028
:1000A00017309F009F0B52289B0B47280000000031
:1000B00000000000000005151A309F009F0B5E280D
:0200C000080036
:02400E00F23F7F
:00000001FF
